:020000040000FA
:0C000000830100308A0004288301372BA4
:10066E0010308312A200A301A401A001AF01B001BA
:10067E00A701A801AB01AC01AD01AE014C30A90040
:10068E001D30AA00103085000730990083169F0197
:10069E0029308500813081008B130B1D542B0B11DB
:1006AE00640083120430850605082939A100A11DB6
:1006BE00622BA301A30A2130A105A2080319712BF5
:1006CE00210824060319702B2108A4001030A20063
:1006DE00712BA203A208031DB82B20082406B1001B
:1006EE00B11EA62BA41E922B2E082D040319892BA6
:1006FE0025082D07A90026080318260A2E07AA008A
:10070E00AD01AE012908AF002A08B000DC30A70009
:10071E000530A800A62B2F082902A5003008031CBF
:10072E00300A2A02A60007302602D030031925020D
:10073E000318A42BAD01AD0AAE01AF01B001200824
:10074E002406B100311CB42B241CB02BFF30AB009F
:10075E00B32B9430AB001130AC001030A200240843
:10076E00A0002E082D040319BF2BAD0A0319AE0AE3
:10077E0030082F040319E32BAF080319B003AF039E
:10078E002F033004031DCF2B2908AF002A08B00019
:10079E002A08B2002908B1002430B1070318B20AA2
:1007AE00FA30B20730083202031DDF2B2F08310258
:1007BE000318E32BA301A30A280827040319ED2B22
:1007CE00A7080319A803A703A301A30A2C082B0447
:1007DE000319F72BAB080319AC03AB03A301A30A50
:1007EE00A3080319FC2B0512FD2B0516A301542B90
:02400E00CC3FA5
:00000001FF
